:02000000012BD2
:20002B0075816331E3111B80FC78FB912EE675F0007B067C009171790C7A009150C001C0C3
:20004B000278F9912EE675F0007B067C00916B79037A059150D007D000C000C007E6898224
:20006B008A8391EC4BD007D000F62278FB912EE675F0007B067C009171790C7A009150C0C5
:20008B0001C00278F9912EE675F0007B067C00916B79037A05915089828A83E493F4D007E8
:2000AB00D000C000C00756D007D000F622E4F508E50875F0007B057C0091C6700801E3E502
:2000CB0008050880EBE508790C7A0075F000915078FB912EE6F701CA227496F509E5097001
:2000EB000801F6E509150980F401EE22E59054C075F000C0E0C0F0E4F5F0790C7A0091507E
:20010B00E7F4D004D0034BC5F04CC5F0F590C29611E4D296E59054C075F000C0E0C0F07465
:20012B000175F000790C7A009150E7F4D004D0034BC5F04CC5F0F590C29711E4D297E5903A
:20014B0054C075F000C0E0C0F0740275F000790C7A009150E7F4D004D0034BC5F04CC5F08D
:20016B00F590C2B711E4D2B7E59054C075F000C0E0C0F0740375F000790C7A009150E7F423
:20018B00D004D0034BC5F04CC5F0F590C2B311E4D2B3E59054C075F000C0E0C0F07404750D
:2001AB00F000790C7A009150E7F4D004D0034BC5F04CC5F0F590C2B211E4D2B222E51185D2
:2001CB0012F091A6F51185F01291AEF9AAF089828A83E49375F00022E4C0E0C0E011B81564
:2001EB008115817401F515E4F519740975F005F51185F01231C8F50BE50B54E075F0007BFB
:20020B00807C0091B570024146E50B541F75F000C333C5F033C5F079247A009150E51185CA
:20022B0012F0F709A7F031C8F50B75F0007BFC7C0091BD7002414441314159E5118512F0FB
:20024B0091AEF51185F012F51385F014415B21FF31C8F50BE50B60024167415BE50B75F096
:20026B00007BC07C0091B57002418A1516E51670024188E5178518F0F51185F012415BE541
:20028B000B75F0007BFD7C0091B5700241AA743F75F000C0E0C0F011B815811581415BE56E
:2002AB000B75F0007BFE7C0091B5700241C6E4C0E0C0E011B815811581415BE50B75F00005
:2002CB007BFF7C0091B5700241E1E5138514F0F51185F012415BE50B75F0007BFC7C0091C0
:2002EB00B57002610F1519E51975F000C333C5F033C5F0791A7A009150E70987F0F5118558
:20030B00F012415BE50B54E06002612A150BE50B75F000C0E0C0F0113415811581415BE56C
:20032B000B54C060026147150BE50B541F75F000C0E0C0F0117615811581415BE50B54A01E
:20034B0060026164150BE50B541F75F000C0E0C0F0113415811581810CE50B30E70261804B
:20036B00150BE50B541F75F000C0E0C0F0117615811581810CE50B54F075F0007BC07C00AA
:20038B0091B5700261A3E50B540FF516E5118512F0F51785F018415BE50B54E075F0007B82
:2003AB00A07C0091B5700261F0E519051975F000C333C5F033C5F0791A7A009150E5118590
:2003CB0012F0F709A7F0E50B541F75F000C333C5F033C5F079247A009150E70987F0F511B9
:2003EB0085F012415BE50B20E702812BE50B75F0007BE07C0091BD7002810CE50B540FF569
:20040B0015E51575F0007B057C009157F50AE50A70088129E50A150A80F411F7811F415BA3
:20042B00415B22C82581C822C92581C97A0022D083D082CF2581F581CFC082C08322CF25CD
:20044B0081F581CF2229F9E5F03AFA22FEEBA4FD8EF0ECA4FCEB8EF0A4C5F02C2DC5F022D6
:20046B0091718EF0ED22C002C001AAF0F97E007D007F11C3E933F9EA33FADF08F5F0E9D0CD
:20048B0001D00222ED33FDEE33FEC3ED9BF5F0EE9C40E0ADF0FED380DB91A604700205F0DB
:2004AB002291AE14B4FF0215F02291E26008E4F5F02291E260F8E4F5F0042291E240F78036
:2004CB00ED91E240F170E780ED91E240E170E780DD91E250E180D7C5F0C39C7003E5F09B82
:2004EB0022FBE493CB22FCE493FB740193CC22FAE493F9740193CA2220041002080180C22D
:20050B00FEE8FDEFC0FC81FE05E2584D42554A5D52475A4F44574C4154495C5146594E4315
:20052B00564B5E53485B50EAEAFC8224E2776C6174697C7166796E63766B7E73687B7065CB
:20054B00786D62756A7D72677A6FEFFC8302E41D441E461C481A4A184C164E145052FC844C
:20056B0022E43D643E663C683A6A386C366E347072FC8501E41B43194517471549134B1132
:20058B004D4FFC8621E43B63396537673569336B316D6FFC8712E41450164E184C1A4A1CE5
:2005AB00481E461D4442FC8832E43470366E386C3A6A3C683E663D6462FC890FE4114D1383
:2005CB004B1549174719451B4341FC8A2FE4316D336B3569376739653B6361FC8B01E442B0
:2005EB00035B045D0559065E085C07570A5A09550C580B530E560D5110544F12EAEAFC8C46
:20060B0021E462237B247D2579267E287C27772A7A29752C782B732E762D7130746F32EAB0
:20062B00FC8D01030507090B0D0F11131517191BFC8E020406080A0C0E10121416181A1C06
:20064B001E1DFC8FC4FEEAADE6AEEEC0FC913C25392842FC902737263E41FC922E363529BE
:20066B004FFC932C382B3352FC943E233B443D21462248244A264C284E2A50B3FC952D318D
:20068B003650342F4E324C304A2E482C462A44B1FC972E2D3154302F563258345A365C380F
:2006AB005E3A5DB1FC9626233B5D21245E225C3D5A3E583C563A54B3FC98393D24433B2227
:2006CB004521472349254B274DB2FC993334304D32314B2F492D472B452943B0FC9B2B30CF
:2006EB0034512D32532F5531573359355BB0FC9A25243D5B22235921573B5539533751B2FD
:20070B00FC9C1E1D0406E5191B0203451C170107481A15094A18130B4C16110D4E140F5012
:20072B0012EAEAFC9D3E3D2426E5393B2223653C372127683A35296A38332B6C36312D6E3E
:20074B00342F7032EAFCA1A0A4AAA3A9EFAFA8A6A7A5EFACE4C1B6B5C0E3C2B6B5C0E2C3B0
:20076B00B6B5C0E1C4B6B5C0E2C3B6B5C0E3C2B6B5C0E4C1B6B5C068666422E8C202E344DC
:20078B0046484A4C4E50525456585A5C5E5D41434547494B4D4F51535557591BEF22E3646B
:2007AB0066686A6C6E70727476787A7C7E7D61636567696B6D6F71737577B0B8BBB8BB77CA
:2007CB00797B21EAC0BCAFBDABAFA2E3C2B4B2B9BAB3B7B0B8B3B5B0BAB3B7C07C7E7D2246
:0F07EB00E8BCAFA8AAA9A3EFBDA5A3EFAFACFFD1
:00000001FF
